:020000040000FA
:020000001228C4
:08000800D000030ED1008312A9
:100010008B1C0B288B1081010B11510E8300D00E0D
:10002000500E09008316FF23900083163F30850091
:10003000283087008312FF308500EE30870083125E
:1000400007309900831600309100831648308100F4
:10005000831231309000831600308C0083121030F0
:100060008B0081018E018F010B118B100B108C0105
:100070000521640087142608013C0319871026080F
:10008000023C0319871007152608013C03190711C4
:100090002608033C031907110518532820150C30B6
:1000A0000F07B100572831080F02031920118719D3
:1000B0005E28A0150C300F07B200622832080F022C
:1000C0000319A011201020192014A010A019A014A9
:1000D0000330871EA006051A72282114C8300F07A6
:1000E000B300762833080F0203192110851A7D28E2
:1000F000A114C8300F07B400812834080F02031977
:10010000A110851888282115C8300F07B5008C2844
:1001100035080F0203192111A1112118A115A118E9
:10012000A1152119A115211221182116A11821129A
:10013000211921120C1C9E280C10B00AA119A32809
:10014000A6010710DB28260803398207AA28B7284A
:10015000C028CE28211CAE280130A600A11CB22840
:100160000330A600211DB6280230A600DB28A11C02
:10017000BB280230A600211DBF280330A600DB28C3
:10018000A11CDB28201CC928071403303007B60047
:10019000CD283608300203190710DB28211DDB2883
:1001A000A01CD728071403303007B600DB28360818
:1001B000300203190710A61CE3282608A700FF3009
:1001C0000F07B700E92837080F02031DE9282608A2
:1001D000A70083169C18032900309B001C141A08E2
:1001E0008312270603190329270883169A00003073
:1001F0009B001C158B1355309D00AA309D009C144C
:100200008B171C11831283123928831600309B0030
:100210001C141A088312A600A700FC39031DA601AE
:10022000A6180714A001A1016400051E2114851E53
:10023000A114851C2115051C2015871DA0156430EF
:100240000F02031D1429FA30B100B200FA30B300D6
:10025000B400B5000130B600FF30B700B0010710A0
:02026000080094
:084000000F000F000F000F007C
:02400E00CC01E3
:024200000000BC
:00000001FF
